:100000000C94340018950000189500001895000015
:10001000189500001895000018950000189500002C
:10002000189500001895000018950000189500001C
:10003000189500001895000018950000189500000C
:1000400018950000189500001895000018950000FC
:1000500018950000189500001895000018950000EC
:1000600018950000189500008FEF8DBFC0EEE8EDE9
:100070004E2E84E08EBFD4E0F4E05F2EEEEFF3E08E
:10008000A0E0B1E0A89584B7082E877F84BF88E1FF
:100090009927809360009093600088278D93319713
:1000A000E9F766243B983A98529853985498219AC5
:1000B000229A81EA8093800084E0809381003D9AB7
:1000C00045983C9A3B9A88E592E0A4E0B1E08D9394
:1000D0009C93E2E0F0E00E94E7000027A9E2B0E094
:1000E0008C9184FB0EF401E041E0041711F00C94B4
:1000F000D9008AEF90E090938B0080938A0086E08D
:1001000090E09093890080938800E2E0F0E00E9404
:10011000E70084E690E00E94F6000027A9E2B0E044
:100120008C9184FB0EF401E041E0041711F00C9473
:10013000B50088EC90E090938B0080938A0084E077
:1001400090E090938900809388008BE090E00E947B
:10015000F6008EE690E090938B0080938A0080E218
:1001600093E00E94F6000C94B5000027A9E2B0E0ED
:100170008C9184FB0EF401E040E0041711F00C9424
:10018000D5008AEF90E0909389008093880086E004
:1001900090E090938B0080938A0080E991E00E9428
:1001A000F6000C946D000C94D5000C948D000C940A
:1001B000E50080E090E0909389008093880080E0E3
:1001C00090E090938B0080938A000C946D0088EEF1
:1001D00093E00CD03197D9F708953197F1F708954E
:1001E000689462F80895E89462F80895EF93FF9395
:1001F000EE27E82BE92B31F0E0EDF7E03197F1F74E
:0A0200000197D1F7FF91EF910895E7
:00000001FF
